:0200000480007A
:100000006F00C004732F2034930F8000630AFF0336
:10001000930F90006306FF03930FB0006302FF038A
:10002000170F0080130F0FFE63040F0067000F000F
:10003000732F203463540F006F00400093E19153FD
:10004000171F000023203FFC6FF09FFF930000006C
:10005000130100009301000013020000930200004E
:100060001303000093030000130400009304000036
:10007000130500009305000013060000930600001E
:100080001307000093070000130800009308000006
:100090001309000093090000130A0000930A0000EE
:1000A000130B0000930B0000130C0000930C0000D6
:1000B000130D0000930D0000130E0000930E0000BE
:1000C000130F0000930F0000732540F1631005002B
:1000D000970200009382020173905230735000180F
:1000E000970200009382020273905230B7020080A0
:1000F0009382F2FF7390023B9302F0017390023AF5
:100100007350403097020000938242017390523046
:10011000735020307350303093010000970200007C
:10012000938282EE73905230130510001315F5017F
:10013000634C05000F00F00F930110009308D005E9
:10014000130500007300000097020080938282EB89
:10015000638A020073905210B7B20000938292102B
:100160007390223073500030372500007320053023
:100170007350300097020000938242017390123452
:10018000732540F17300203017250000072085E714
:1001900017250000872045E7D3F00010532510A055
:1001A000930310009301200063147506530510A0FB
:1001B0009303100093013000631C7504531510A0C5
:1001C000930300009301400063147504537000D042
:1001D00013051000D37005D0D3F00010532510A0E4
:1001E000930310009301500063147502530510A08F
:1001F0009303100093016000631C7500531510A059
:1002000093030000930170006314750063103002C3
:100210000F00F00F638001009391110093E1110032
:100220009308D00513850100730000000F00F00F44
:10023000930110009308D00513050000730000001F
:04024000731000C077
:1010000000000000000000000000000000000000E0
:1010100000000000000000000000000000000000D0
:1010200000000000000000000000000000000000C0
:1010300000000000000000000000000000000000B0
:081040000000000000000000A8
:10200000000080FF000040400000000000000000D1
:040000058000000077
:00000001FF
